:10F800005542200135D0085A824506023140800217
:10F810003F4004000F9308249242060220012F83E8
:10F820009F4F18F90002F8233F4002000F9307246E
:10F830009242060220011F83CF430402F923B24003
:10F84000805A2001C2435600D242FF105700D242D4
:10F85000FE105600F2D006005800F2D04000220000
:10F86000F2D040002600B24071027201B240100294
:10F870006001B240F00064018243740132D018008C
:10F880000F4332D0F000FD3F304016F90F120E1238
:10F890000D120C12B2F0FEFF64011D4200020F4D6A
:10F8A0008F104F4F12C30F100E4F1E531C420402F5
:10F8B0000F4C1F53824F04021CF30B203F90F401A6
:10F8C00013341F4202020D5F824D00022F53824FFC
:10F8D00002021F4270010E9FFC2F824E74013C41B8
:10F8E0003D413E413F4100133F90E8030D341F422C
:10F8F00002022F83824F02020D8F824D00021F42AF
:10F9000070010E9FE62FE93F824304021F427001FF
:08F910000E9FDF2FE23F001300
:04F9180001000300E7
:10FFE00088F888F888F888F888F888F888F888F811
:10FFF0008CF888F888F888F888F888F888F800F885
:040000030000F80001
:00000001FF
